:100000000C9423040C948F040C9441080C948F04DA
:100010000C94B8090C948F040C948F040C948F04E6
:100020000C948F040C948F040C948F040C94A01DDA
:100030000C948F040C94F02B0C948F040C948F046C
:100040000C948F040C948F040C948F040C94452C06
:100050000C948F040C948F040C948F040C948F04D4
:100060000C948F040C948F040C948F040C948F04C4
:100070000C948F04FC0C0A0D160D160DEE0C160DCB
:10008000160D160D160D160D160D160D160D160D58
:10009000160D160D160D160DF00C160DF20C160D94
:1000A000160D160D160D0E0D160D250D0C0D160D3B
:1000B000160D160D160D160D160D160D160D160D28
:1000C000160D160D160D160DE60C020DF40C060D90
:1000D000160DF60C160DFA0C160D040DF80C080D85
:1000E000FE0C000D160D160D160D160D160D160D27
:1000F000160DE80CEA0CEC0C100D120D160D160D79
:10010000160D140DC00DC20DCE0DCE0DCE0DCE0DA3
:10011000CE0DCE0DC40DC60DC80DCE0DCE0DC20D2B
:10012000D10DCE0DCE0D8A0DC00DCE0DCE0DC60D4E
:10013000CE0DCE0DCE0DCE0DCE0DCE0DC80DC00DFB
:10014000AC0DCE0DB00DCE0DCE0DCE0D8C0DC40D63
:10015000CE0DCE0DBA0DCE0DCE0DCE0D8E0DCC0D1D
:10016000CE0DAE0DCE0DC20DCE0DCE0DBE0DB20D0F
:10017000CE0DB40DC60DCE0DCE0DCE0DBC0DB60DF3
:10018000CE0DCE0DCE0DCE0DCE0DCE0DCE0DB80DAD
:10019000CE0D900DCE0DCE0DC40DCE0DCE0DCC0DD1
:1001A000CE0DCE0DCE0DCE0DCE0DCE0DCE0DCE0D77
:1001B000CE0D920DCE0DCE0DCE0DBA0DCE0DCE0DB7
:1001C000CE0DCE0DCE0DCE0DCE0DCE0DCE0DCE0D57
:1001D000940DCE0D960D980DCE0DCE0DCE0D9A0D23
:1001E0009C0D9E0DCE0DA00DA20DCE0DCE0DCE0DF3
:1001F000CA0DA40DCE0DA80DA60DAA0DCE0DCE0DC7
:10020000CE0DCE0DCC0D130E610E3C0E870EAD0E35
:10021000B50EBC0EC10EC50E5C0F5E0F600F620FF7
:10022000640F6C0F6C0F6C0F660F680F6A0F441031
:10023000651079109610A810B310D710F010161191
:1002400038110E12B3139115061C2D1C251D2D1CE3
:10025000251D791C9C1C251DF31C021DCD21CD21C3
:10026000052205228022B422AB24AB24CB22AB246E
:100270005C225C226524AB247A24982472253032D7
:10028000582000522000643A25752000633A2575F5
:1002900020006973723A25303458200077253032B7
:1002A000582000214353335F4630210A0021435335
:1002B000335F5245414459210A00214353335F5271
:1002C00045534554210A00214353325F45305F4670
:1002D00030210A00214353325F463021202530323D
:1002E000580A00214353325F4530210A002143530D
:1002F000325F494E4954210A00214353315F453052
:100300005F25303258210A004D5B783A2564207908
:100310003A256420763A256420683A256420623ABA
:10032000253032585D0A000A5B434C525D20004C78
:10033000257520000A4D6F7573653A2025730A00F4
:100340000A4445463A20000A4558503A20000A49D6
:100350004E543A20000A4C4F473A20000A4C4D5365
:100360003A200053257520000A49443A2530345874
:1003700028257325732920000A556E6B6E6F776EE2
:100380002049443A205265706F727420746F205473
:100390004D4B20004E4720004F4B20000A3535378B
:1003A000365F43533832683A00522575200057258E
:1003B0007520005725752000572575200058257594
:1003C0002000412575200049257520005B434847E2
:1003D0005D20000A2575205052543A2530325820AD
:1003E0004953523A2530345820005B5253545D2013
:1003F000000A2575204552523A253032582049537B
:10040000523A253034582000535B2530325820258D
:1004100030325820253032585D2000007B460102E2
:1004200003763A687F6577482B353B69787964397C
:10043000141E3C6A7A1D16041A1F3D6B061B070822
:1004400021203E6C2C19091715223F6D11050B0A4E
:100450001C23406E7E100D182425416F360E0C12A1
:100460002726427037380F33132D43717534322FDE
:100470002E44727C7D28303174457351504A524D60
:10048000492A5466594F5C5F4C4B4E62635A5D5E1D
:1004900060295367585B56576147554842403E3C78
:1004A0003A3B456843413F3D2B357E697A79007878
:1004B000141E7C6A7B1D16041A1F7F6B061B07081F
:1004C00021204D6C2C19091715224A6D11050B0AB4
:1004D0001C234C6E49100D182425516F360E0C123A
:1004E00027264F7037380F33132D52717534502F24
:1004F0002E4E72397D283065314B735464586776BF
:10050000012A773259745C5F66020362635A5D5E4A
:1005100060295344575B565561474680291E1F206A
:10052000212223242526272D2E2A2B141A081517BD
:100530001C180C12132F302878041607090A0B0D0B
:100540000E0F33343579311D1B061905111036375E
:10055000387D557A2C393A3B3C3D3E3F4041424341
:1005600053475F6061565C5D5E57595A5B626346F4
:1005700048644445677B7F650301025250514F68D0
:10058000696A6B6C6D6E6F7071725800494C754A78
:100590004D734B4E767C777E7466540A4C6F6F7049
:1005A0002073746172742E0A000A55534220636FDF
:1005B0006E666967757265642E0A000A544D4B3A7F
:1005C0003464366537662F4C5546413A6436613798
:1005D00064660A003403490042004D0020005000C8
:1005E000430020006B006500790062006F0061002D
:1005F00072006400200063006F006E0076006500EA
:1006000072007400650072000000080354004D0081
:100610004B0000000403090409025B00030100A071
:100620003209040000010301010009211101000148
:10063000223900070581032000010904010001039C
:10064000010200092111010001227F000705820338
:100650000800010904020002030000000921110141
:100660000001222200070583032000010705030380
:100670002000011201100100000008EDFEEE1B0138
:1006800002010200010631FF0974A101097515007C
:1006900026FF009520750881020976150026FF00C7
:1006A000952075089102C005010902A1010901A167
:1006B000008501050919012908150025019508750E
:1006C0000181020501093009311581257F950275E7
:1006D00008810609381581257F9501750881060571
:1006E0000C0A38021581257F950175088106C0C066
:1006F00005010980A10185021601002637001A8133
:10070000002AB700751095018100C0050C0901A1F0
:10071000018503160100269C021A01002A9C02751D
:100720001095018100C005010906A101050719E026
:1007300029E71500250195087501810205081901B1
:10074000290595057501910295017503910105072C
:10075000190029F71500250195F875018102C0637C
:100760006F6E73756D65723A20253034580A0073C8
:10077000797374656D3A20253034580A000A0025D3
:1007800030325820006B6579626F6172643A2000E4
:100790004C45443A20253032580A0025583A253035
:1007A00031366225730A000A202030313233343565
:1007B000363738394142434445460A0064656C5F28
:1007C0006B65795F6269743A2063616E2774206497
:1007D000656C3A20253032580A006164645F6B65AD
:1007E000795F6269743A2063616E27742061646482
:1007F0003A20253032580A00290A002575002F00BA
:100800002575005D28002564002000256400200077
:1008100025640020002564007C0025303258006DDE
:100820006F7573656B6579205B62746E7C78207977
:10083000207620685D287265702F61636C293A20EC
:100840005B002F0BF41511241FBECFEFD4E0DEBFE9
:10085000CDBF04B603FE41C08091210490912204D3
:10086000A0912304B09124048730904BA740B04B53
:10087000A1F51092210410922204109223041092E8
:10088000240414BE0FB6F894A89580916000886186
:1008900080936000109260000FBE109201081092C9
:1008A0000008E3E0F0E089E080935700E491E695EA
:1008B000E370E150E33040F4F0E0EE0FFF1FE85842
:1008C000FE4F8081918102C080E090E1E0E0F0E89D
:1008D000E81BF90BF695E795099511E0A0E0B1E06A
:1008E000E4E7F1E602C005900D92AE37B107D9F703
:1008F00024E0AEE7B1E001C01D92A132B207E1F7FA
:1009000014E0C3E2D4E004C02197FE010E949E30AF
:10091000C132D107C9F70E9423190C94B8300C9446
:100920000000FF93EF93E0917E01F0917F013097FB
:1009300009F00995EF91FF910895FC0185918030B0
:1009400011F0EFDFFBCF0895FF27E0E230E247FF31
:100950000CC0419597FF09C0EDE2609570958095B8
:100960009095611D711D811D911D27FF02C021956C
:1009700030E350E2AA27660F771F881F991FAA1F2E
:10098000A41710F0A41B63955A95A9F7AA3008F094
:10099000A95FA05DAF93F395611571058105910580
:1009A00041F7ED3211F4EF93F395F21718F43F93FA
:1009B000F395FBCF8F91B5DFFA95E1F70895E991B3
:1009C000F9918591803021F0853219F0AADFF9CFB5
:1009D000089520E0E89455915532C1F3503311F455
:1009E000689455915A3348F4505390F3220F022ED5
:1009F000220F220F200D250FF4CF0EF4219589919F
:100A00009991533619F3533729F1533559F1BC01F4
:100A100088279927E8945C3621F489919991689404
:100A20005591543639F446EF7EF077FF0DC08FEFC5
:100A30009FEF0AC055374AE039F0583540E121F0C0
:100A4000523642E009F00895FF93EF937DDFEF9176
:100A5000FF91B7CFFF93EF93FC0181918030B9F301
:100A600060DFFBCFFF93EF9368DFF1CFDF93CF938E
:100A7000CDB7DEB72596A3DFCF91DF910895FC01B6
:100A80002AB1938D909592239AB99BB1838D892B2E
:100A90008BB90895FC019AB1838D809589238AB919
:100AA0009BB1838D892B8BB985E08A95F1F7000086
:100AB00099B1838D982381E009F480E00895FC01C9
:100AC0002BB1948D909592239BB99AB1848D892BEB
:100AD0008AB90895FC012AB1948D909592239AB910
:100AE0009BB1848D892B8BB90895FC019AB1848DBB
:100AF000809589238AB99BB1848D892B8BB985E038
:100B00008A95F1F7000099B1848D982381E009F46A
:100B100080E008950F931F93CF93DF938C01EB0137
:100B2000C8010E944A05882341F0209731F085E0F2
:100B30008A95F1F700002197F3CFCE01DF91CF9195
:100B40001F910F9108950F931F93CF93DF938C0103
:100B5000EB01C8010E944A05811108C0209731F0BD
:100B600085E08A95F1F700002197F3CFCE01DF9160
:100B7000CF911F910F9108950F931F93CF93DF9300
:100B80008C01EB01C8010E947505811108C02097F6
:100B900031F085E08A95F1F700002197F3CFCE017F
:100BA000DF91CF911F910F910895CF93DF93EC01C7
:100BB0000E943F05CE01DF91CF910C946A053BB1B5
:100BC000FC01238D209523232BB93AB1238D232BB0
:100BD0002AB90C946A05FC018CB3938D982B9CBBAD
:100BE0009DB3838D892B8DBB0895CF93DF93EC014B
:100BF0000E94EB05CE01DF91CF910C94D505FC014D
:100C00002DB3938D909592239DBBCF010C94DF055E
:100C1000FC01118210821282138280E090E8958399
:100C20008483178210860895CF93DF93EC012E986A
:100C300026982F9827980E94DF05898D843080F4AC
:100C400040916900880F22E030E0B90102C0660FD0
:100C5000771F8A95E2F7CB01842B8093690010C03F
:100C600040916A008370880F22E030E0B90102C031
:100C7000660F771F8A95E2F7CB01842B80936A0079
:100C80009DB38B8D809589238DBBCE01DF91CF9154
:100C90000C940806CF93DF93EC018F8190E00196CE
:100CA0008F709927288530E08217930749F4CE0189
:100CB0000E940806CE010E94EB05CE010E94D505D8
:100CC0002FB7F89498858F81891751F0FE01E90FAD
:100CD000F11D81859F5F9F709887C82FD0E002C06B
:100CE000CFEFDFEF2FBFCF3F8FEFD80781F080919D
:100CF000060480FF0CC0DF93CF938CE792E09F93B4
:100D00008F930E9436050F900F900F900F90CE0199
:100D1000DF91CF9108950F931F93CF938C01CAE178
:100D2000C15071F0C8010E944A068F3F2FEF920711
:100D300049F48FE99FE00197F1F700C00000F0CF80
:100D40008FEF9FEFCF911F910F9108952F923F92B8
:100D50004F925F926F927F928F929F92AF92BF92CB
:100D6000CF92DF92EF92FF920F931F93CF93DF9377
:100D7000EC01062F1B828091060480FF0CC01F929D
:100D80006F938CE992E09F938F930E9436050F90AA
:100D90000F900F900F908C819D818115904891F05C
:100DA0008091060480FF0EC08C819D819F938F935C
:100DB00082E992E09F938F930E9436050F900F90E7
:100DC0000F900F908C819D8181159048D9F7CE01AD
:100DD0000E944A05811115C08091060480FF11C050
:100DE00068EE73E0CE010E94A3059F938F938CE879
:100DF00092E09F938F930E9436050F900F900F9073
:100E00000F90CE010E947505811115C080910604D6
:100E100080FF11C068EE73E0CE010E94BC059F9375
:100E20008F9386E892E09F938F930E9436050F90F0
:100E30000F900F900F909DB38B8D809589238DBB64
:100E40009BE0D92ECC24C39410E09924939428E0FD
:100E5000222E37E0332E46E0842E55E0752E64E0D6
:100E6000662E73E0572EE2E04E2EF3E8AF2EF2E04E
:100E7000BF2ECE010E94DF058FE193E00197F1F7CD
:100E800000C00000CE010E945F058FE193E0019752
:100E9000F1F700C00000CE010E943F0560E177E25B
:100EA000CE010E948A05892B11F49B826AC0E12C35
:100EB000F12C90E59A95F1F7C8010E2C02C095959A
:100EC00087950A94E2F780FF05C0C924CE010E94ED
:100ED0006A0503C0CE010E945F0562E370E0CE01A7
:100EE0000E94A305892B11F44B824BC062E370E092
:100EF000CE010E948A05892B11F45B8242C02FEF3C
:100F0000E21AF20A88E0E816F10499F690E59A955B
:100F1000F1F7CE01CC2019F00E946A0502C00E94B0
:100F20005F0562E370E0CE010E94A305892B11F4F6
:100F30006B8227C062E370E0CE010E948A05892B94
:100F400011F47B821EC020E52A95F1F7CE010E94A4
:100F50006A058CE2E82EFF24F394CE010E94750509
:100F6000882329F0E114F104D9F58B820AC0EF2817
:100F7000E1F36CE271E0CE010E94BC05892B49F4DB
:100F80003B828B81813009F03FC0DA94D11030C0B0
:100F90003BC06CE271E0CE010E94A305892B11F4E5
:100FA0002B82EFCFCE010E940806CE010E94D5050C
:100FB000CE010E94EB05CE01DF91CF911F910F91E1
:100FC000FF90EF90DF90CF90BF90AF909F908F9069
:100FD0007F906F905F904F903F902F900C948B0676
:100FE00085E08A95F1F7000091E0E91AF108B5CFA4
:100FF0001B828091060480FF3CCFBF92AF920E947B
:1010000036050F900F9035CF8B8180618B83CE0199
:101010000E94DF058FE39FE10197F1F700C0000018
:10102000CE010E94D505CE010E94EB058FEF9FEF08
:10103000DF91CF911F910F91FF90EF90DF90CF90B4
:10104000BF90AF909F908F907F906F905F904F90E8
:101050003F902F9008951F93CF93DF93EC01162FAD
:101060006DEE0E94A6068A3F910539F4612FCE01EC
:10107000DF91CF911F910C94A606DF91CF911F9124
:1010800008951F920F920FB60F9211242F933F9342
:101090004F935F938F939F93EF93FF9349B1509139
:1010A000B701909107042091A1013091A20121156F
:1010B000304819F49093A3010FC08091A301981BAD
:1010C000933050F08091A1019091A20190939E01E4
:1010D00080939D0180E21EC12091A1013091A20167
:1010E000369527953093A2012093A10181E090E0ED
:1010F00001C0880F5A95EAF7842349F08091A10135
:101100009091A20190689093A2018093A101809197
:10111000A1019091A20199278038910509F41BC182
:10112000A8F48032910509F416C138F4009709F447
:1011300012C1409709F495C0B5C08034910509F4F7
:101140000AC18035910509F48CC0ACC0803C910582
:1011500031F148F48039910509F483C0803A910552
:1011600009F44DC09FC0803D910509F47AC0803ECE
:10117000910509F097C08091A1019091A2019093EF
:101180009E0180939D018091A1019091A201892FE0
:1011900099279093A2018093A10183E256C0809188
:1011A0009F01811123C084E629B19091B801922357
:1011B00011F48111B8C029B19091B8019223E1F0E6
:1011C0008111B7C08091A1019091A20190939E01DD
:1011D00080939D018091A1019091A201892F99276F
:1011E0009093A2018093A10182E22FC080919F0180
:1011F000823209F0B0C0E6CF8111ADC0E3CF80915B
:101200009F01811125C084E629B19091B8019223F4
:1012100011F4811194C029B19091B8019223F1F099
:10122000811193C08091A1019091A20190939E01A0
:1012300080939D018091A1019091A201892F99270E
:101240009093A2018093A10181E280939F0136C017
:1012500080919F01813209F07EC0E4CF81117BC073
:10126000E1CF8091A1019091A20190939E01809382
:101270009D018091A1019091A20197FF02C080E1A0
:1012800001C081E180939F018091A1019091A20111
:1012900026E0969587952A95E1F79093A201809391
:1012A000A1010CC010929F018091A1019091A20117
:1012B00090939E0180939D0180E82CC02091A10114
:1012C0003091A2018091A401E82FF0E0E356FE4F97
:1012D00021878F5F8F708093A40190E001968F70BB
:1012E00099273091A501432F50E08417950769F4A1
:1012F0002DB38091B801482F409524232DBB9BB17D
:1013000094239BB99AB1892B8AB98091A401831344
:1013100003C080E48093A00180E090E89093A20154
:101320008093A10118C095E09A95F1F700008150D3
:101330003BCF95E09A95F1F7000081503CCF95E0C6
:101340009A95F1F7000081505FCF95E09A95F1F7FB
:101350000000815060CFFF91EF919F918F915F913D
:101360004F913F912F910F900FBE0F901F901895A6
:101370001F920F920FB60F9211242F933F934F930A
:101380005F938F939F93EF93FF9349B150919A018D
:1013900090910704209184013091850121153048F6
:1013A00019F4909386010FC080918601981B9330A9
:1013B00050F08091840190918501909381018093F8
:1013C000800180E21EC12091840130918501369513
:1013D0002795309385012093840181E090E001C03E
:1013E000880F5A95EAF7842349F0809184019091FF
:1013F0008501906890938501809384018091840198
:101400009091850199278038910509F41BC1A8F4B2
:101410008032910509F416C138F4009709F412C11D
:10142000409709F495C0B5C08034910509F40AC10C
:101430008035910509F48CC0ACC0803C910531F138
:1014400048F48039910509F483C0803A910509F484
:101450004DC09FC0803D910509F47AC0803E910542
:1014600009F097C08091840190918501909381014A
:10147000809380018091840190918501892F992723
:10148000909385018093840183E256C0809182010C
:10149000811123C084E629B190919B01922311F41C
:1014A0008111B8C029B190919B019223E1F0811183
:1014B000B7C08091840190918501909381018093C0
:1014C00080018091840190918501892F99279093C3
:1014D00085018093840182E22FC080918201823253
:1014E00009F0B0C0E6CF8111ADC0E3CF8091820199
:1014F000811125C084E629B190919B01922311F4BA
:10150000811194C029B190919B019223F1F0811136
:1015100093C0809184019091850190938101809383
:1015200080018091840190918501892F9927909362
:1015300085018093840181E28093820136C080918D
:101540008201813209F07EC0E4CF81117BC0E1CFFE
:101550008091840190918501909381018093800115
:10156000809184019091850197FF02C080E101C0C4
:1015700081E180938201809184019091850126E030
:10158000969587952A95E1F790938501809384013C
:101590000CC01092820180918401909185019093FA
:1015A00081018093800180E82CC0209184013091DA
:1015B000850180918701E82FF0E0E058FE4F2187F8
:1015C0008F5F8F708093870190E001968F709927CD
:1015D00030918801432F50E08417950769F42DB3AB
:1015E00080919B01482F409524232DBB9BB19423D0
:1015F0009BB99AB1892B8AB980918701831303C063
:1016000080E48093830180E090E89093850180934B
:10161000840118C095E09A95F1F7000081503BCF06
:1016200095E09A95F1F7000081503CCF95E09A95AE
:10163000F1F7000081505FCF95E09A95F1F7000037
:10164000815060CFFF91EF919F918F915F914F916A
:101650003F912F910F900FBE0F901F901895EDE9BD
:10166000F1E0118210821282138220E030E835838B
:101670002483168291E0918F128E82E0838F948F63
:10168000E0E8F1E011821082128213823583248314
:10169000168293E0918F828F88E0838F84E0848F1D
:1016A0000895E62FF0E034E0F595E7953A95E1F7F7
:1016B000E7706F70823079F08330C1F0813011F5BE
:1016C000F0E024E0EE0FFF1F2A95E1F7E60FF11D91
:1016D000E55EFA4F15C0F0E094E0EE0FFF1F9A951B
:1016E000E1F7E60FF11DE556FB4F0AC0F0E084E09C
:1016F000EE0FFF1F8A95E1F7E60FF11DE55EFB4F48
:101700008491089580E808950F931F93CF93DF93FA
:101710008C01EB0169EEFC01808191810E94A6069B
:10172000F801808191810E948B068883F801808175
:1017300091810E948B068983F801808191810E94AA
:101740008B068A8399279F938F9389811F928F930A
:1017500088811F928F9388E094E09F938F930E94DB
:1017600036058DB79EB708960FB6F8949EBF0FBE8C
:101770008DBFDF91CF911F910F910895E6EDF1E0BC
:101780001192119281E0E63EF807D1F708951F9378
:10179000CF93DF93FC0184810E94510B87FD20C011
:1017A000182F1F70C82FD0E094E0D595C7959A9553
:1017B000E1F7612F8C2F0E94E71F811111C0CC0F20
:1017C000DD1FCA52DE4F81E090E002C0880F991FF2
:1017D0001A95E2F728813981822B932B998388838C
:1017E000DF91CF911F9108951F93CF93DF93FC0159
:1017F00084810E94510B87FD22C0182F1F70C82FB3
:10180000D0E094E0D595C7959A95E1F7612F8C2F9C
:101810000E94E71F882399F0CC0FDD1FCA52DE4FCC
:1018200081E090E002C0880F991F1A95E2F7809539
:101830009095288139818223932399838883DF912E
:10184000CF911F9108958091C8019091C9010E9484
:1018500014068091BA019091BB010C9414068091FA
:1018600006048160809306040C94BE0BE82FF0E020
:10187000EE0FFF1FEA52FE4F8081918108950C9474
:10188000BE0BE82FF0E083E0EE0FFF1F8A95E1F733
:101890007770E70FF11D94E0EE0FFF1F9A95E1F7C7
:1018A0006F70E60FF11DEE0FFF1FE050F8498591B4
:1018B00094910895FC018481823070F0843061F04D
:1018C00062FB992790F960FD926061FD9460692F39
:1018D000808191810C942B080895CF93C82F682F95
:1018E00088EC91E00E945A0C6C2F8AEB91E0CF912A
:1018F0000C945A0CCF92DF92EF92FF920F931F93AA
:10190000CF93DF936C018B010E941E2C7C01F601AA
:10191000808191810E944A06EC01019631F4C70151
:101920000E94362C8017910790F3CE01DF91CF9162
:101930001F910F91FF90EF90DF90CF9008950F933C
:101940001F93CF93DF93FC0180819181DC0112967C
:101950002C912131F9F08F0162EF0E94A6068F3F92
:10196000BFEF9B07D1F08A3F9105D1F464EF71E09E
:10197000C8010E947A0C8F3F2FEF9207A1F0D82F59
:10198000CC2764EF71E0C8010E947A0CDE01A82B1D
:10199000CD010BC08DEF9FEF08C08FEF9FEF05C00B
:1019A0008EEF9FEF02C080E090E0DF91CF911F911A
:1019B0000F910895CF93862F90E0FC017C97E83437
:1019C000F105A0F5E65CFF4F0C949E3085E53EC026
:1019D0008AE53CC08BE53AC08CE538C08DE536C061
:1019E0008EE534C08FE532C080E630C081E62EC07F
:1019F00082E62CC083E62AC08FE628C081E726C095
:101A000082E724C084E722C085E720C087E71EC0A4
:101A100088E71CC08AE71AC08CE718C08FE716C099
:101A200080E714C089E712C08BE710C0C62F1F9251
:101A30006F9389EF92E09F938F930E9436050F90EA
:101A40000F900F900F908C2F01C084E5CF910895D7
:101A5000CF93DF93EC0199859230A9F128F4992373
:101A600041F09130C9F045C09330B1F19430D9F1D3
:101A700040C0603E21F0613E21F482E02BC081E055
:101A800029C067FD04C0CE010E94C70B33C06F7729
:101A9000CE010E94F40B2EC0663359F118F46A325D
:101AA00029F427C06A3A29F1663B19F167FD05C0A0
:101AB000CE010E94DA0C682F12C06F77CE010E940F
:101AC000DA0C682F13C06D3121F06D3991F484E088
:101AD00001C083E089870EC0653459F465E5CE0105
:101AE0000E94C70B06C0653C21F465E5CE010E944B
:101AF000F40B198680E0DF91CF910895862F90E056
:101B0000FC013397E138F10508F048C0EE57FF4F6C
:101B10000C949E3087E108958FE108958CE5089537
:101B200080E6089582E6089587E2089583E50895A2
:101B30008FE2089589E3089587E308958FE3089578
:101B400087E408958FE4089586E508958EE5089565
:101B50008FE7089580E0089585E608958EE608955C
:101B60008FE6089580E3089588E3089580E408955A
:101B700088E4089580E5089587E508958FE5089540
:101B800088E1089588E0089580E2089580E108954D
:101B900089E108958DE6089588E20895862F8F776C
:101BA00008958FE008956B35C9F068F46131F1F064
:101BB00020F46E30C9F484E50895633169F064352A
:101BC00099F48BE508956D3559F050F0623651F077
:101BD0006C3751F487E7089581E108958DE5089504
:101BE0008AE608958EE00895862F08958FE008957F
:101BF000613131F0613411F48CE70895862F089536
:101C000083E108951F93CF93DF93EC01162FEA85AC
:101C10008E2F90E08930910508F0BDC0FC01ED5F8A
:101C2000FE4F0C949E308A819B8180599B4A02977B
:101C300020F4CE010E94D30D182F103E69F030F42D
:101C4000133871F0143871F46FE792C0113E31F01F
:101C5000103F41F481E093C082E091C084E08FC0E6
:101C600062E086C01A8617FD02C0612F21C00E9463
:101C7000BE0B8DEE92E069C08A819B8180599B4AA0
:101C8000029720F4CE010E94F80D182F193509F49F
:101C900082C0103F19F0123119F47DC083E06FC08B
:101CA0001A8617FD09C0612FCE010E947E0D682F94
:101CB000CE010E94C70B70C00E94BE0B83EE92E063
:101CC00044C08A819B8180599B4A029720F4CE01AF
:101CD0000E94D30D182F133821F0143821F46FE728
:101CE00057C062E055C01A8617FD02C0612F25C09B
:101CF0000E94BE0B1F921F9384ED92E09F938F93DF
:101D00000E9436050F900F900F900F9024C08A818B
:101D10009B8180599B4A029720F4CE010E94F80DC6
:101D2000182F1A861231C1F11935B1F117FD09C00A
:101D3000612FCE010E947E0D682FCE010E94F40B10
:101D40002BC00E94BE0B87EC92E09F938F930E9462
:101D500036050F900F908FEF20C0643121F0603F67
:101D6000D1F486E00CC085E00AC06737A1F460E0DA
:101D7000CE010E94C70B0FC0643169F487E08A87E7
:101D80000BC0603F41F488E0FACF673721F460E090
:101D9000CE010E94F40B1A8680E0DF91CF911F9153
:101DA00008956C3551F018F4633169F00AC0663754
:101DB00031F06E3731F486E7089581E508958EE7B6
:101DC0000895862F08958DE50895CF93DF93EC0154
:101DD0006F3B41F028F486E5860F823070F402C034
:101DE0006C3F59F41B868AEB92E09F938F930E947D
:101DF00036050F900F908FEFB1C08B85813009F4BD
:101E000045C038F0823009F476C0833009F491C0BF
:101E1000A4C08A819B8182399B4A21F4CE010E9411
:101E2000D10E682F663809F168F46338D1F020F4D8
:101E3000603819F582E077C06438A9F06538E9F4B4
:101E400068E61DC06C38A9F030F4673881F06B3853
:101E5000A1F461E014C06D3871F0603F71F481E06D
:101E600062C062E00CC06FE70AC068E708C060E0CB
:101E700006C069E004C06AE002C067FD04C0CE018C
:101E80000E94C70B6AC08DEA92E02EC01B868A8131
:101E90009B8182399B4A21F4CE010E94D10E682F8A
:101EA000862F90E0FC01E358F109EB30F105A0F436
:101EB000E45FFE4F0C949E3062E010C06FE70EC0EE
:101EC00068E60CC068E70AC060E008C061E006C0D0
:101ED00069E004C06AE002C067FD04C0CE010E9450
:101EE000F40B3BC083EA92E09F938F930E943605E8
:101EF0000F900F9032C0653279F030F4663171F096
:101F00006E3199F460E00BC0663221F0603F69F4F5
:101F100083E009C06DE503C063E501C061E5CE0162
:101F20000E94C70B04C08B8718C00E94BE0B1B8683
:101F300014C06E3169F020F46631B9F761E509C06B
:101F4000653221F0663289F76DE503C063E501C0B3
:101F500060E0CE010E94F40BEACF80E0DF91CF91E8
:101F600008958F929F92AF92BF92CF92DF92EF929D
:101F7000FF920F931F93CF93DF9300D000D01F9257
:101F8000CDB7DEB78C01DC01ED91FC918381882314
:101F9000B1F1E080F180D3800E941E2CFF92EF927D
:101FA0001F92DF929F938F9381EF93E09F938F9384
:101FB0000E943605D801ED91FC91119783818075BF
:101FC0000FB6F894DEBF0FBECDBF81F418968C918A
:101FD0008B3061F48AEE93E09F938F930E943605D5
:101FE0008CE0D80118968C930F900F90D801ED914A
:101FF000FC9111971382ED91FC9111821082D8010E
:10200000ED91FC9111978281882381F1928115963F
:102010008C91981759F1E080F180D2800E941E2C9B
:10202000FF92EF921F92DF929F938F9383ED93E045
:102030009F938F930E943605F80185810FB6F8941F
:10204000DEBF0FBECDBF0190F081E02D85FF03C044
:10205000928194FD6FC584FD6AC5D801ED91FC9114
:102060001197828115968C9311821082D80118964F
:10207000EC918E2F90E08D30910508F09AC5FC010F
:10208000E95EFE4F0C949E300E941E2C9F938F930E
:1020900087EC93E09F938F930E943605F80114829A
:1020A0001382128215820E94BE0B0E941E2CD80140
:1020B00017969C938E93169781E018968C93189799
:1020C0008D919C910E94F5056DC0F80180819181F0
:1020D0000E944A060196C9F7D80116968D919C91E7
:1020E00017970E94362C893B9B4008F462C582E01A
:1020F00018C00E941E2C9F938F9382EC93E09F93B5
:102100008F930E9436056FEFD8018D919C910E94AC
:10211000A6060F900F900F900F908A3F910521F423
:1021200086E0F801808745C583E060C3F8018081BF
:1021300091810E94FF052E98269A2F98279A0E9437
:102140001E2CD80117969C938E93169784E04FC34C
:10215000F801868197810E94362C853F914008F4D2
:1021600028C585E043C32E9826982F982798F80114
:10217000808191810E940806D8018D919C910E94D6
:10218000F5050E941E2C9F938F938DEB93E09F93F8
:102190008F930E9436050E941E2CF8019783868338
:1021A00086E080870F900F900F900F9002C5D801A6
:1021B0008D919C910E944A06019609F4FAC40E94EE
:1021C0001E2C9F938F9388EB93E09F938F930E9495
:1021D00036050E941E2CF8019783868387E0E1CFA5
:1021E000D80116968D919C9117970E94362C853FA9
:1021F000914018F089E0F8018087D8018D919C9179
:102200000E944A06019609F4D4C40E941E2C9F9392
:102210008F9383EB93E09F938F930E9436050E94E8
:102220001E2CF8019783868388E0BBCFD8011696D1
:102230008D919C9117970E94362C853F914018F004
:1022400089E0F8018087D8018D919C910E944A060F
:10225000019609F4AEC40E941E2C9F938F938EEAC0
:1022600093E09F938F930E94360589E0F80199CF00
:10227000C8010E949F0CD80113969C938E931297CD
:102280000E941E2C9F938F9389EA93E09F938F93D4
:102290000E943605F801828193810F900F900F9074
:1022A0000F90009711F482E010C08F3FBFEF9B07A3
:1022B00011F481E044C09C012D5F3F4F2230310575
:1022C00090F38F3F910529F484E0D80114968C9304
:1022D00063C09C0125583B4A2230310508F445C4AF
:1022E0008239BBEA9B0709F440C49C0120593B4A50
:1022F00022303105F8F48CE993E09F938F930E948C
:10230000360560EFF801808191810E94A6060F904A
:102310000F908A3F910509F01FC462E8D8018D91A2
:102320009C910E94A6068A3F910509F015C488E990
:1023300093E014C4803BBFEB9B0721F483E0F801DA
:1023400084832AC088278115FBEA9F0709F4ABCF55
:1023500081152FEB920791F381159F4779F388E759
:1023600093E09F938F930E94360560EFD8018D9183
:102370009C910E94A6060F900F908A3F910509F04C
:10238000F4C362E0F801808191810E94A6068A3F31
:10239000910509F0EAC387CFF801228133812E3FEE
:1023A000FFEF3F0751F02D3F4FEF340749F0211564
:1023B000310549F040E251E008C041E251E005C07A
:1023C0004BE151E002C047E251E0D80114968C91F4
:1023D000813049F0823051F0833059F0843061F01F
:1023E0008CE391E00BC080E391E008C08DE291E0C6
:1023F00005C083E391E002C081E491E05F934F93D5
:102400009F938F933F932F9388E693E09F938F93AF
:102410000E9436058AE0F80180877DC30E941E2C49
:102420009F938F9383E693E09F938F930E9436054B
:102430000F900F900F900F90D80114968C918330CD
:1024400031F0843079F0823009F07CC106C068EF49
:10245000F801808191810E94A6060E946B1E0E9455
:102460006D0C70C165EFD8018D919C910E94A606FC
:102470006AEEF801808191810E94A606BE016F5F1D
:102480007F4FC8010E94840B8CE593E09F938F934C
:102490000E94360568EED8018D919C910E94A60697
:1024A00060E0F801808191810E94A60666EED80165
:1024B0008D919C910E94A60666EEF8018081918123
:1024C0000E94A60666EED8018D919C910E94A606F8
:1024D000BE016F5F7F4FC8010E94840B0F900F9069
:1024E0008981882309F47AC08A81882309F476C017
:1024F00085E593E09F938F930E94360566EEF80181
:10250000808191810E94A60668EED8018D919C91F0
:102510000E94A60660E0F801808191810E94A606D3
:1025200068EED8018D919C910E94A60663E0F801A7
:10253000808191810E94A60668EED8018D919C91C0
:102540000E94A60662E0F801808191810E94A606A1
:1025500068EED8018D919C910E94A60661E0F80179
:10256000808191810E94A60666EED8018D919C9192
:102570000E94A60668EEF801808191810E94A6065D
:1025800063E0D8018D919C910E94A60668EEF80147
:10259000808191810E94A60661E0D8018D919C9175
:1025A0000E94A60668EEF801808191810E94A6062D
:1025B00062E0D8018D919C910E94A60668EEF80118
:1025C000808191810E94A60663E0D8018D919C9143
:1025D0000E94A60689E0F801848781C08EE493E01A
:1025E0009F938F930E94360563EFD8018D919C9144
:1025F0000E94A60668ECF801808191810E94A606DF
:1026000063EFD8018D919C910E94A60664E6F801C3
:10261000808191810E94A60663EFD8018D919C91E3
:102620000E94A60660E5F801808191810E94A606BD
:10263000C8010E949F0C292F30E00F900F9023308B
:10264000310511F080E001C083E0D8011C968C9325
:1026500087E493E09F938F930E94360563EFF80120
:10266000808191810E94A60668ECD8018D919C9191
:102670000E94A60663EFF801808191810E94A60660
:1026800068ECD8018D919C910E94A60663EFF80139
:10269000808191810E94A60660E5D8018D919C9170
:1026A0000E94A606C8010E949F0C292F30E00F90BF
:1026B0000F902430310511F080E001C084E0F80172
:1026C000848781110EC080E493E09F938F930E94D2
:1026D000360566EFD8018D919C910E94A6060F9059
:1026E0000F9064EFF801808191810E94A606BE01DF
:1026F0006F5F7F4FC8010E94840BD8011C968C919C
:10270000893049F0833051F0843059F0882361F0EA
:1027100083E291E00BC08FE491E008C087E491E090
:1027200005C088E591E002C081E691E09F938F9318
:1027300084E393E09F938F930E9436050F900F9050
:102740000F900F908BE0F80180870E941E2C9F93C2
:102750008F938FE293E09F938F930E9436050F90A3
:102760000F900F900F90D8018D919C910E944A0676
:102770004C01019609F41DC2F8018481843069F18D
:102780008114910421F0FFEF8F16910469F40E94E7
:10279000BE0B0E947D2187E293E09F938F930E945E
:1027A00036050F900F9005C2823069F0833081F0BA
:1027B000813009F0FEC1682DC8010E94280D8F3FAD
:1027C00009F0F7C112C0682DC8010E94020EF7CFB0
:1027D000682DC8010E94E50EF2CFF8018081918139
:1027E0000E948B066C01019629F48CE0D8011896A2
:1027F0008C93DFC1F801808191810E948B067C015E
:10280000019699F3D8011C968C91FE0131965F01D7
:10281000853028F4833030F4882321F0DCC08930FF
:10282000A1F0D9C0D8011D969C911D97987F282DA5
:102830002770922B1D969C9384FE02C0DD24DA94AF
:1028400085FEC4C0FF24FA94C1C0F8013585C401D7
:10285000887499278834910509F0A9C0C1FEA7C0E2
:10286000F0E38F229924959487949594879420E39C
:10287000C222DD2454E0D594C7945A95E1F7C828C4
:10288000D92842E0C416D104E1F183E0C816D1048E
:1028900009F476C0CA94CD2809F07CC1E6FC17C0C3
:1028A000A701487055278E2D8F70E7FE07C0452B76
:1028B00011F420E001C020EF822B0AC0452B11F457
:1028C00020E001C020EF982F922B80E002C080E032
:1028D00090E0E4FE05C03860D8011D963C9303C02B
:1028E000377FF8013587D8011D962C911D97E5FE9D
:1028F00004C020611D962C934FC12F7EF8012587BF
:102900004BC1E0FE05C03064D8011D963C9303C066
:102910003F7BF8013587D8011D968C911D97E1FE0C
:1029200004C080681D968C9303C08F77F80185875B
:10293000D8011D968C911D97E2FE04C080621D9601
:102940008C9303C08F7DF8018587D8011D968C91EB
:102950001D97E3FE04C080641D968C9303C08F7B9B
:10296000F8018587D8011D968C911D97E4FE04C05F
:1029700080681D968C930EC18F77F80185870AC1F8
:10298000C70124E0959587952A95E1F7E7FE03C0F6
:10299000806F90E003C0982F9F7080E0387F2E2DCD
:1029A0002770E32EE22AD8011D96EC92F5C0387FFD
:1029B000882D8770382BF801358784FE02C0DD240E
:1029C000DA9485FE4DC0FF24FA944AC0833049F062
:1029D0008430C9F045C0833079F4E12CF12CC12C4E
:1029E000D12CD8018D919C910E948B068F3FBFEF17
:1029F0009B07B1F1982F35C0843009F0CBC0E12C92
:102A0000F12CC12CD12CF801808191810E948B0680
:102A1000AC018F3FFFEF9F0719F183FD02C080E0FB
:102A200001C080EF942F9F70982BD8011D962C9198
:102A30001D9744FF04C028601D962C9303C0277F78
:102A4000F8012587D8011D962C911D9745FF04C0DC
:102A500020611D962C9305C02F7EF801258701C0AB
:102A600090E085E0D5011D928A95E9F7F80185850A
:102A7000898380E0F0E8CF16D1044CF4960141E858
:102A8000C4164FEFD40624F421E83FEF01C02FE72E
:102A90002A83A0E8EA16F10454F49701B1E8EB1692
:102AA000BFEFFB0614F421E83FEF219501C021E8B8
:102AB0002B83903811F0919501C09FE79C8380385B
:102AC00009F481E88D83C5010E94C01E89811F928F
:102AD0008F938D81282F082E000C330B3F938F93FB
:102AE0008C81282F082E000C330B3F938F938B8102
:102AF000282F082E000C330B3F938F938A81282FA9
:102B0000082E000C330B3F938F9388E093E09F9344
:102B10008F930E9436050FB6F894DEBF0FBECDBF6F
:102B200048C00E947D21D80118961C9242C0828123
:102B300085FF93CAD80118968C918B3009F08DCA05
:102B40008CEC93E09F938F930E9436058CE0F80104
:102B500080870F900F9081CA84E993E09F938F93B1
:102B60000E9436050F900F909ECB60EFF801808198
:102B700091810E94A6068A3F910509F094CB63E0FB
:102B8000D8018D919C910E94A6068A3F910509F07B
:102B90008ACBD4CB80E090E025E0D5011D922A9528
:102BA000E9F7F80125852983E12CF12CC12CD12CE2
:102BB00065CF81E00F900F900F900F900F90DF91F5
:102BC000CF911F910F91FF90EF90DF90CF90BF902A
:102BD000AF909F908F90089588EC91E00E94B10F84
:102BE0008AEB91E00C94B10FE8ECF1E08DE991E013
:102BF000918380831382128214821582108611863B
:102C000012861386148615860E94BE0BEAEBF1E04D
:102C100080E891E09183808313821282148215826E
:102C20001086118612861386148615860C94BE0BA8
:102C300080910A030895CF93DF9300D01F92CDB700
:102C4000DEB720911804243021F523E029839B83EB
:102C50008A8382E08093E9008FEF9091E8008150B1
:102C600095FD06C095ED9A95F1F700008111F5CF1D
:102C70008091E80085FF0DC040E050E063E070E027
:102C8000CE0101960E94D71A8091E8008E7780933A
:102C9000E8000F900F900F90DF91CF910895CF93A0
:102CA000DF9300D01F92CDB7DEB7209118042430F7
:102CB00061F519821A821B8222E0298381389105ED
:102CC00020F0805891099B838A8382E08093E900F9
:102CD0008FEF9091E800815095FD06C095ED9A9593
:102CE000F1F700008111F5CF8091E80085FF0DC05C
:102CF00040E050E063E070E0CE0101960E94D71AF8
:102D00008091E8008E778093E8000F900F900F90ED
:102D1000DF91CF91089520911804243051F522E0DD
:102D20002093E9002FEF3091E800215035FD06C0D7
:102D300035ED3A95F1F700002111F5CF2091E8002B
:102D400025FF17C020911001222341F021E020939C
:102D5000F10040E050E065E070E004C040E050E089
:102D600063E070E00E94D71A8091E8008E7780932C
:102D7000E8000895CF93DF9320911804243009F0E0
:102D80004AC0EC01809111018823E1F08091120189
:102D90008823C1F081E08093E90081E8815049F007
:102DA0009091E80095FD05C09AE29A95F1F700C070
:102DB000F5CF8091E80085FF2EC040E050E060E252
:102DC00070E019C081E08093E90081E8815059F0FA
:102DD0009091E80095FD07C0EFE3F1E03197F1F73E
:102DE00000C00000F3CF8091E80085FF14C040E0F0
:102DF00050E068E070E0CE010E94D71A8091E800B0
:102E00008E778093E80080E2FE01AAEEB2E00190A6
:102E10000D928A95E1F7DF91CF910895CF93C091FC
:102E2000E801C1110BC00E942A2C643C7940810545
:102E3000910520F081E08093E801C1E08C2FCF91D3
:102E40000895FF920F931F93CF93DF93D82F0FB660
:102E500007FE83C080911804843081F080910301C3
:102E600090E001962091050130E082239323209188
:102E7000040130E08217930709F0C9C00E940E17C1
:102E8000811110C08091030190E00196209105010D
:102E900030E0822393232091040130E082179307CE
:102EA00009F0B5C00E941E2C8C01C091E900CF70C2
:102EB0009091EC00892F817090FD80E8C82B83E011
:102EC0008093E90085E0F82E8091EB0085FD42C0FB
:102ED0008091EB0080FF3EC08091EE0087FF3AC0FA
:102EE0008091040190910301981709F457C09091C3
:102EF000E80095FF8AC0E0910101F0910201E80F1E
:102F0000F11D20818F5F9091050189238093040139
:102F10002093F1008091E80085FDE2CF8091E800E8
:102F200080FFDECF8091E8008E778093E800F092FA
:102F30000001D6CF8091030190E001962091050118
:102F400030E0822393232091040130E0821793071D
:102F500009F448C0CF70C093E90040910301842F69
:102F600090E001962091050130E082239323209187
:102F7000040130E08217930709F44CC0E09101018D
:102F8000F0910201E40FF11DD083809103018F5F66
:102F9000909105018923809303013CC08091E80052
:102FA00085FF33C0D093F10081E09091F200992326
:102FB00091F09091E80090FF0EC09091E80095FF8D
:102FC00003C01092F100F9CF9091E8009E779093A2
:102FD000E800F0920001882309F4ACCFCF70C093D1
:102FE000E90018C080910001882309F4B3CF0E9442
:102FF0001E2C9C018017910711F4890165CF9091D7
:103000000001915090930001F8CF80E0CECF409125
:103010000301B4CF80E0DF91CF911F910F91FF901A
:103020000895089542E261EC81E00E94501A42E066
:1030300061EC82E00E94501A42E261EC83E00C9461
:10304000501A80911A04833009F453C030F481304F
:1030500071F0823009F4BAC008958A3009F4A6C02C
:103060008B3009F478C0893009F0C8C020C0809145
:103070001904813A09F0C2C08091E800877F8093EB
:10308000E80080911D0490911E04892B21F460E2D8
:103090008AEE92E003C060E080E090E070E00E9481
:1030A000241B8091E8008B778093E800089580913D
:1030B0001904813209F0A2C080911D0490911E0470
:1030C000892B09F09BC08091E800877F8093E800FE
:1030D0008091E80082FD05C0809118048111F8CF2D
:1030E0008DC08091F10080930A038091E8008B7776
:1030F00081C080911904813A09F080C080911D043B
:1031000090911E04892BA1F48091E800877F809321
:10311000E8008091E80080FFFCCF8091110180934E
:10312000F1008091E8008E778093E8000E94851A74
:1031300080911D0490911E04019709F05FC0809159
:10314000E800877F8093E8008091E80080FFFCCF53
:10315000809110014AC080911904813209F04EC05B
:1031600080911D0490911E04892B69F48091E800E0
:10317000877F8093E8000E94851A80911B048093CA
:1031800011010E947D2180911D0490911E040197E0
:10319000A9F58091E800877F8093E8000E94851A56
:1031A00080911B04809310010C947D21809119045F
:1031B000813221F58091E800877F8093E8000E94AA
:1031C000851A80911C0480930B0308958091190443
:1031D000813AA1F48091E800877F8093E800809194
:1031E000E80080FFFCCF80910B038093F100809179
:1031F000E8008E778093E8000C94851A08958091FA
:103200000A038093E90110920A030E943F0C0C9478
:103210007D210C94FF180E94CA2B809116048823EC
:1032200029F00E94D72B81110C943A1A08950E941C
:10323000EC2B8091E90180930A0308950C941719EF
:1032400008950C942019CF9384B7877F84BF0FB65D
:10325000F894A89580916000886180936000109236
:1032600060000FBE90E080E80FB6F8948093610094
:10327000909361000FBE81E297E10E94892B86E066
:1032800091E00E94661E8BEB95E00E949D040E94D7
:10329000230C0E94251F0E943D1D0E94901D7894C2
:1032A0000E94271F80911804843029F00E944B1E31
:1032B0000E942019F7CF89EA95E00E949D040E94A0
:1032C00021198BE995E00E949D04C3E080911804C8
:1032D000853019F40E940B19F9CF0E94B32B0E947C
:1032E0002B1F2091E4003091E5008091E601909140
:1032F000E7012817390709F464C08091E400909130
:10330000E5009093E7018093E6010E940E17882361
:1033100009F457C080911804843009F052C080919C
:10332000E9008F702091EC00922F917020FD90E8C1
:10333000892BC093E9009091EB0090FF3FC09091E2
:10334000EE0097FF3BC090910401209103012917E3
:1033500009F12091E80025FF1DC0E0910101F091E5
:103360000201E90FF11D30819F5F20910501922339
:10337000909304013093F1009091E80095FDE3CF24
:103380009091E80090FFDFCF9091E8009E779093B6
:10339000E800D9CF9091F200992381F09091E80054
:1033A00090FF0CC09091E80095FF03C01092F100CF
:1033B000F9CF9091E8009E779093E8008F7080930A
:1033C000E9000E944B1E82CF292F3327233031057D
:1033D000C9F060F42130310581F02230310509F067
:1033E00041C08BE590E028E136E040C02132310554
:1033F000E1F02232310531F135C082E190E023E77E
:1034000036E034C099278130910549F028F00297C1
:1034100049F5E4EDF5E005C0E4E1F6E002C0EAE0DC
:10342000F6E0849190E09F0121C063307105D0F4F3
:10343000660F771FFB01EE58FE4F2081318189E036
:1034400090E014C06330710568F4FB01EE0FFF1FBC
:10345000E459FE4F20813181FB01E759FE4F808105
:1034600090E004C080E090E020E030E0FA01318399
:103470002083089584E089BD86E089BD09B400FEFB
:10348000FDCF8091D8008F7D8093D8008091E0009F
:1034900082608093E0008091E00081FDFCCF089580
:1034A000982F953068F59093E900981739F070914E
:1034B000EC002091ED005091F00003C0242F762FF6
:1034C00050E021FD02C09F5FECCF3091EB003E7FCA
:1034D0003093EB003091ED003D7F3093ED00309163
:1034E000EB0031603093EB007093EC002093ED0023
:1034F0005093F0002091EE0027FDE5CF80E0089585
:103500008F708093E90081E008958091190487FF0E
:1035100011C08091E80082FD05C0809118048111DE
:10352000F8CF11C08091E8008B770BC08091180410
:10353000882349F08091E80080FFF8CF8091E8006F
:103540008E778093E80008952091E4003091E500A3
:1035500095E64091EC00842F817040FF23C080915C
:10356000E80080FD1DC080911804882399F0853003
:1035700099F08091EB0085FD11C04091E4005091DD
:10358000E5002417350729F3915011F09A01E1CF96
:1035900084E0089582E0089583E0089581E008952D
:1035A00080E008954091E80042FFDDCF0895CF927A
:1035B000DF92EF92FF920F931F93CF93DF93EC0173
:1035C0008B017A010E94A41A811135C0E114F10423
:1035D00039F0F70180819181081B190BC80FD91FA1
:1035E000C12CD12C0115110529F18091E80085FD30
:1035F00018C08091E8008E778093E8000E944B1EEF
:10360000E114F10449F0F70180819181C80ED91EBF
:10361000D182C08285E00FC00E94A41A882311F3D2
:103620000AC089918093F10001501109FFEFCF1A70
:10363000DF0AD8CF80E0DF91CF911F910F91FF90EB
:10364000EF90DF90CF90089520911F0430912004D7
:103650002617370748F06115710539F42091E80005
:103660002E772093E80001C0B901FC0120E061152C
:10367000710561F1809118048823D9F18530D9F161
:103680008091E80083FD39C08091E80082FD2BC065
:103690008091E80080FFEBCF8091F20090E061150F
:1036A000710551F08830910538F421912093F10093
:1036B000615071090196F3CF21E0089709F020E0ED
:1036C0008091E8008E778093E800D1CF2111D2CF8E
:1036D0000AC080911804882361F0853061F08091E0
:1036E000E80083FD0AC08091E80082FFF2CF80E00D
:1036F000089582E0089583E0089581E0089520917F
:103700001F04309120042617370748F06115710512
:1037100039F42091E8002E772093E80001C0B90128
:10372000FC0120E06115710579F18091180488236E
:1037300009F43DC0853009F43CC08091E80083FD68
:103740003AC08091E80082FD2CC08091E80080FFA3
:10375000E9CF8091F20090E06115710559F0883051
:10376000910540F424912093F10031966150710944
:103770000196F2CF21E0089709F020E08091E8005F
:103780008E778093E800CECF2111CFCF0AC08091F1
:103790001804882361F0853061F08091E80083FD92
:1037A0000AC08091E80082FFF2CF80E0089582E0B5
:1037B000089583E0089581E008951F93CF93DF93E8
:1037C000CDB7DEB7AA970FB6F894DEBF0FBECDBF58
:1037D000E9E1F4E08091F100819324E0E132F20725
:1037E000C9F70E9421188091E80083FF2EC18091C3
:1037F000190490911A04492F50E04A30510508F0FD
:1038000024C1FA01EC5DFE4F0C949E30803821F00B
:10381000823809F01AC108C08091150490911604ED
:10382000992389F082600FC080911D048F708530CC
:1038300008F00BC18093E9008091EB0085FB88279D
:1038400080F91092E9009091E800977F9093E8004A
:103850008093F1001092F100D1C0282F2D7F09F044
:10386000F4C0882319F0823061F0EFC080911B040E
:10387000813009F0EAC0933009F080E080931604AB
:103880002EC080911B0481112AC080911D048F706D
:103890002FEF280F243008F0D8C08093E900209142
:1038A000EB0020FF1CC0933021F48091EB0080627C
:1038B00014C09091EB0090619093EB0021E030E018
:1038C000A90102C0440F551F8A95E2F74093EA0010
:1038D0001092EA008091EB0088608093EB001092D8
:1038E000E9008091E800877F8093E8000E94851AB4
:1038F000ACC08111AAC010911B041F778091E30016
:103900008078812B8093E3008091E800877F80930B
:10391000E8000E94851A8091E80080FFFCCF80912A
:10392000E30080688093E300111102C082E001C0CF
:1039300083E08093180489C08058823008F085C0E5
:1039400080911B0490911C048C3D53E0950779F500
:1039500083E08A838AE289834FB7F894DE01139665
:1039600020E03EE051E2E32FF0E050935700E49175
:1039700020FF03C0E295EF703F5FEF708E2F90E065
:10398000EA3010F0C79601C0C0968D939D932F5FCB
:10399000243149F74FBF8091E800877F8093E8008A
:1039A0006AE270E0CE0101960E94241B16C060916D
:1039B0001D0470911E04AE014F5F5F4F0E94E41919
:1039C000BC01892B09F441C09091E800977F909346
:1039D000E80089819A810E947F1B8091E8008B77A3
:1039E0008093E80032C0803881F58091E800877FBD
:1039F0008093E800809114048093F1008091E800A6
:103A00008E7772CF811121C080911B0490911C048C
:103A100099270297D4F48091E800877F8093E8008B
:103A200080911B04809314040E94851A80911404D1
:103A3000811106C08091E30087FD02C081E001C0D2
:103A400084E0809318040E9412188091E80083FF9C
:103A50000AC08091E800877F8093E8008091EB00A6
:103A600080628093EB00AA960FB6F894DEBF0FBE7B
:103A7000CDBFDF91CF911F9108950E949A1D0E94A2
:103A80009D1DE0EEF0E0808181608083E8EDF0E054
:103A900080818F77808319BCE3E6F0E080818160CC
:103AA00080831092170408950E949A1D0E949D1D04
:103AB0008091D8008F778093D8008091D80080685B
:103AC0008093D8008091D8008F7D8093D80084E0C7
:103AD00089BD86E089BD09B400FEFDCF10921804AF
:103AE00010921404109216041092150442E060E043
:103AF00080E00E94501A8091E1008E7F8093E10067
:103B00008091E20081608093E2008091E200886011
:103B10008093E2008091E0008E7F8093E000089522
:103B2000E3E6F0E080818E7F808381E0809317045C
:103B30000C94541D1092E20008951092E100089533
:103B40001F920F920FB60F9211242F933F934F9312
:103B50005F936F937F938F939F93AF93BF93EF93F5
:103B6000FF938091E10082FF0BC08091E20082FF11
:103B700007C08091E1008B7F8093E1000E944A1E84
:103B80008091E10080FF19C08091E20080FF15C0A4
:103B90008091E2008E7F8093E2008091E20080615C
:103BA0008093E2008091D80080628093D80019BC95
:103BB00085E0809318040E9409198091E10084FF38
:103BC00030C08091E20084FF2CC084E089BD86E093
:103BD00089BD09B400FEFDCF8091D8008F7D809310
:103BE000D8008091E1008F7E8093E1008091E20017
:103BF0008F7E8093E2008091E20081608093E200FA
:103C000080911404882311F084E007C08091E300C0
:103C100087FD02C081E001C083E0809318040E9408
:103C20001E198091E10083FF24C08091E20083FF90
:103C300020C08091E100877F8093E10082E0809343
:103C40001804109214048091E1008E7F8093E100AB
:103C50008091E2008E7F8093E2008091E20080619B
:103C60008093E20042E060E080E00E94501A0E94EF
:103C70001118FF91EF91BF91AF919F918F917F911B
:103C80006F915F914F913F912F910F900FBE0F90C9
:103C90001F9018950895CF93809118048823A1F060
:103CA000C091E900CF709091EC00892F817090FD58
:103CB00080E8C82B1092E9008091E80083FD0E9403
:103CC000DD1BCF70C093E900CF910895909311034D
:103CD000809310030895E0911003F0911103309741
:103CE00021F00190F081E02D099480E00895EF9299
:103CF000FF920F931F93CF93DF93E0911003F09106
:103D000011033097B1F18C010280F381E02D099508
:103D10008091060482FF2DC080FF04C085E897E0F3
:103D20000E949D04E80110E28FE7E82E87E0F82E5C
:103D30008091060480FF0BC088811F928F93FF92B1
:103D4000EF920E9436050F900F900F900F90115038
:103D500021961111EDCF8091060480FF0AC08DE7F6
:103D600097E0DF91CF911F910F91FF90EF900C940E
:103D70009D04DF91CF911F910F91FF90EF900895D7
:103D8000E0911003F0911103309721F00480F58148
:103D9000E02D09940895CF93DF9320910E03309185
:103DA0000F032817390709F190930F0380930E032F
:103DB000E0911003F09111033097B9F0EC01068007
:103DC000F781E02D09958091060482FF0EC080FFE7
:103DD0000CC0DF93CF938FE697E09F938F930E9461
:103DE00036050F900F900F900F90DF91CF910895AF
:103DF000CF93DF9320910C0330910D0328173907DF
:103E000009F190930D0380930C03E0911003F0915E
:103E100011033097B9F0EC010084F185E02D09958C
:103E20008091060482FF0EC080FF0CC0DF93CF9309
:103E30008FE597E09F938F930E9436050F900F9028
:103E40000F900F90DF91CF9108950C94E61F0E9480
:103E5000152C0C942F0C8F929F92AF92BF92CF9201
:103E6000DF92EF92FF920F931F93CF93DF9300D0D7
:103E700000D01F92CDB7DEB70E94EC1503E113E02E
:103E8000F12C8F2D0E94360C4C01F801A080B180DE
:103E9000A826B926A114B10439F4F3940E5F1F4F7C
:103EA000F8E0FF12EECF39C08091060481FD0E9438
:103EB000FA1FE12CCC24C394D12CC5018C219D2167
:103EC000892B21F1E982FA8221E0C4018C219D2114
:103ED000892B09F420E02B830E941E2C8160782F0F
:103EE0009D838C8349815A816B818D810E94302012
:103EF00049815A816B817C818D810E94B52BF801AB
:103F0000808191818C259D2591838083E394CC0CC5
:103F1000DD1CF0E1EF12D1CFC0CF8FEF89838A8310
:103F20001B820E941E2C8160782F9D838C83498187
:103F30005A816B818D810E9430200E94B42B0E9497
:103F40008E2E0E946B1E90911203891759F10E94C8
:103F50006B1E809312039091060492FF0EC090FF97
:103F60000CC01F928F9380E997E09F938F930E94DC
:103F700036050F900F900F900F90809112030F90C5
:103F80000F900F900F900F90DF91CF911F910F9195
:103F9000FF90EF90DF90CF90BF90AF909F908F9069
:103FA0000C94C62B0F900F900F900F900F90DF91F5
:103FB000CF911F910F91FF90EF90DF90CF90BF9026
:103FC000AF909F908F9008950C946D0C0895CF93AF
:103FD000C62F0E94360C21E030E002C0220F331FB2
:103FE000CA95E2F72823392381E0232B09F480E0E6
:103FF000CF910895EF92FF920F931F93CF93DF938A
:1040000087EA97E00E949D04C0E0D0E080E2E82EBD
:1040100081E0F82E0BE917E08C2F0E94360C0E94ED
:10402000A02BFF92EF929F938F93DF93CF931F93D9
:104030000F930E94360521968DB79EB708960FB64E
:10404000F8949EBF0FBE8DBFC830D10529F7DF9110
:10405000CF911F910F91FF90EF90089508950895CB
:10406000CF93DF93CDB7DEB72B970FB6F894DEBFB3
:104070000FBECDBF942F4F83252F588769877A872E
:104080008B874A855B85452B31F02F3F31F481E0EA
:104090009F3F19F403C081E001C080E080FD07C0AC
:1040A0004F81588569857A858B850E94B52BDE0105
:1040B000119686E0FD0111928A95E9F785E0FE01EF
:1040C000379601900D928A95E1F749815A816B816B
:1040D0007C818D819E810E949A272B960FB6F89441
:1040E000DEBF0FBECDBFDF91CF910895882309F4C5
:1040F000BBC09CEF980F913A18F40E94842A0DC01F
:1041000090E2980F983058F4877091E001C0990FB1
:104110008A95EAF7892F0E94292B0C94632B9BE543
:10412000980F933070F4853A29F0863A31F083E89D
:1041300090E005C081E890E002C082E890E00C9435
:10414000CB1E98E5980F973108F08EC0883A09F495
:1041500045C0893A09F445C08A3A09F445C08B3A0A
:1041600009F445C08C3A09F445C08D3A09F445C0BC
:104170008E3A09F445C08F3A09F445C0813B09F4F1
:1041800045C0803B09F445C0823B09F445C0833BF0
:1041900009F445C0843B09F445C0853B09F445C09A
:1041A000863B09F445C0873B09F445C0883B09F4C8
:1041B00045C0893B09F445C08A3B09F445C08B3BA7
:1041C00009F445C08C3B09F445C08D3B09F445C05A
:1041D0008E3B09F445C080E090E044C082EE90E060
:1041E00041C089EE90E03EC08AEE90E03BC085EB96
:1041F00090E038C086EB90E035C083EB90E032C0B1
:1042000084EB90E02FC087EB90E02CC08CEC90E02A
:1042100029C08DEC90E026C083E891E023C08AE8B5
:1042200091E020C082E991E01DC084E991E01AC0CC
:1042300081E292E017C083E292E014C084E292E04F
:1042400011C085E292E00EC086E292E00BC087E2E8
:1042500092E008C08AE292E005C08FE690E002C0DA
:1042600080E790E00C94F81E0895882329F19CEFD4
:10427000980F913A18F40E94D42A0DC090E2980F3A
:10428000983058F4877091E001C0990F8A95EAF749
:10429000892F0E942F2B0C94632B9BE5980F933052
:1042A00020F480E090E00C94CB1E885A873120F4F3
:1042B00080E090E00C94F81E0895882321F00E947D
:1042C000292B0C94632B0895882321F00E942F2B17
:1042D0000C94632B08950E94492B0E94182B0E9476
:1042E000632B0E94342F0E94012E80E090E00E94F8
:1042F000CB1E80E090E00C94F81E0E94392B0C94A9
:104300006B21CF92DF92EF92FF920F931F93CF9387
:10431000DF9300D000D01F92CDB7DEB76C010E94B2
:10432000C82B811118C385E0F601DE0111960190BA
:104330000D928A95E1F7F601408151812381348104
:104340002115310531F05F3F31F481E04F3F19F421
:1043500003C081E001C080E080FDFDC2F601F28073
:10436000E580E2948FE0E82249835A83FB82722F32
:104370003D832C836F2D8D810E94F9298C010E9431
:10438000F8290E94F228E12FE295EF708E2F90E03D
:10439000FC01E25DFE4F0C949E30812F807F1F70E8
:1043A000882311F01295107FFF20B9F0112329F016
:1043B000812F0E943C2B0E94632B802F0F900F9027
:1043C0000F900F900F90DF91CF911F910F91FF9061
:1043D000EF90DF90CF900C947620802F0E943521B3
:1043E000112309F4B8C2812F0E94422B0F900F9025
:1043F0000F900F900F90DF91CF911F910F91FF9031
:10440000EF90DF90CF900C94632B812F807F1F70F3
:10441000803211F01295107F002319F0013009F15C
:104420002BC0FF20A9F0EE2059F1F1E0812FEF120F
:1044300028C00F900F900F900F900F90DF91CF91A9
:104440001F910F91FF90EF90DF90CF900C944C2B29
:10445000EE2021F021E0E21609F47DC20E944F2BEC
:104460004DC0FF20E9F085E08E1508F474C20E946B
:10447000262B812329F042C0FF20F1F1E11015C065
:10448000812F0F900F900F900F900F90DF91CF9191
:104490001F910F91FF90EF90DF90CF900C945D21D2
:1044A00094E09E1508F457C229C0F601858180FF6B
:1044B00013C08F708583E4CF003F09F489C108F0F1
:1044C00055C180E4800F803208F459C1FF2009F4FF
:1044D000EAC1EE2009F49AC1802F0E9476200933A8
:1044E00009F0DAC1FFEF21EE84E0F1502040804076
:1044F000E1F700C000002FC2E110D7C1812F59C1E0
:10450000812F86958695837019F08130B9F023C28A
:10451000FF2019F0C801937002C080E090E00F9076
:104520000F900F900F900F90DF91CF911F910F91EF
:10453000FF90EF90DF90CF900C94CB1EFF2019F0EE
:10454000C801937002C080E090E00F900F900F9030
:104550000F900F90DF91CF911F910F91FF90EF90EF
:10456000DF90CF900C94F81E802FFF2019F00E944E
:10457000142D02C00E947C2D0F900F900F900F9071
:104580000F90DF91CF911F910F91FF90EF90DF90EF
:10459000CF900C94012E812F837009F070C0F11020
:1045A000DAC1202F229526952770220F220F602F27
:1045B0006F70862F90E0A0E0B0E06C017D01022ECC
:1045C00004C0CC0CDD1CEE1CFF1C0A94D2F704FFC7
:1045D00012C08FE090E0A0E0B0E004C0880F991F07
:1045E000AA1FBB1F2A95D2F7BC01CD01609570951B
:1045F0008095909503C060E070E0CB01169516950C
:1046000013701230B1F040F56C297D298E299F2955
:10461000113031F10F900F900F900F900F90DF91AC
:10462000CF911F910F91FF90EF90DF90CF900C945E
:104630000D296C297D298E299F290F900F900F90AD
:104640000F900F90DF91CF911F910F91FF90EF90FE
:10465000DF90CF900C9427290E940D29C701B60145
:104660000F900F900F900F900F90DF91CF911F91AF
:104670000F91FF90EF90DF90CF900C94F328FF20E4
:1046800019F0812F817001C08695882309F463C1D8
:10469000202F229526952770220F220F602F6F70F2
:1046A000862F90E0A0E0B0E06C017D01022E04C0F6
:1046B000CC0CDD1CEE1CFF1C0A94D2F704FF12C0C8
:1046C0008FE090E0A0E0B0E004C0880F991FAA1F1F
:1046D000BB1F2A95D2F7BC01CD01609570958095DE
:1046E000909503C060E070E0CB01169516951370AD
:1046F0001230B1F040F56C297D298E299F291130A7
:1047000031F10F900F900F900F900F90DF91CF919C
:104710001F910F91FF90EF90DF90CF900C94D429D0
:104720006C297D298E299F290F900F900F900F9053
:104730000F90DF91CF911F910F91FF90EF90DF903D
:10474000CF900C94E6290E94D429C701B6010F909E
:104750000F900F900F900F90DF91CF911F910F91BD
:10476000FF90EF90DF90CF900C94C229023F09F4A4
:104770005EC008F449C0033F09F46CC0A7CE902F77
:104780009071E92E812F8F71FF2051F00E945B29DB
:10479000802FEE2019F08295807F73CE8F7071CEBE
:1047A0000E947C29802FEE2019F08295807F01C025
:1047B0008F700F900F900F900F900F90DF91CF910F
:1047C0001F910F91FF90EF90DF90CF900C94642198
:1047D000FF20A9F0E4E0EE1508F4BDC0812F8F7131
:1047E0000F900F900F900F900F90DF91CF911F912E
:1047F0000F91FF90EF90DF90CF900C94A129F5E0FE
:10480000FE1508F4A8C0EACFFF2099F0812F8F7120
:104810000F900F900F900F900F90DF91CF911F91FD
:104820000F91FF90EF90DF90CF900C945B29FF20C9
:1048300069F3812F8F710F900F900F900F900F9051
:10484000DF91CF911F910F91FF90EF90DF90CF906C
:104850000C947C29FF2089F0812F8F710F900F908D
:104860000F900F900F90DF91CF911F910F91FF90BC
:10487000EF90DF90CF900C9446290F900F900F90FF
:104880000F900F90DF91CF911F910F91FF90EF90BC
:10489000DF90CF900C944129033509F423CE0734DF
:1048A00009F059C01FCEEE2021F2802F0F900F90FB
:1048B0000F900F900F90DF91CF911F910F91FF906C
:1048C000EF90DF90CF900C943521412F4F70602FE7
:1048D000C6010E948A2C0F900F900F900F900F909E
:1048E000DF91CF911F910F91FF90EF90DF90CF90CC
:1048F0000C944D2801112FC0FF2069F10E947D21E9
:104900002FEF80E792E0215080409040E1F700C017
:1049100000000F900F900F900F900F90DF91CF91AC
:104920001F910F91FF90EF90DF90CF900C946B2C24
:10493000412F4F70602FC6010F900F900F900F9076
:104940000F90DF91CF911F910F91FF90EF90DF902B
:10495000CF900C948D2C0F900F900F900F900F9084
:10496000DF91CF911F910F91FF90EF90DF90CF904B
:1049700008951F93CF93DF9300D000D01F92CDB73F
:10498000DEB7942F4983252F5A836B837C838D83D5
:104990004C815D81452B31F02F3F31F481E09F3F09
:1049A00019F403C081E001C080E0182F117080FD70
:1049B00024C049815A816B817C818D810E94F929B3
:1049C000292F22952F702C3030F42A3048F42250B1
:1049D000223068F013C02C3061F02F3051F00EC03F
:1049E000803C28F0803E50F0815F833038F011E049
:1049F00005C093FB112710F901C010E0812F0F9023
:104A00000F900F900F900F90DF91CF911F9108950D
:104A1000CF93DF9300D000D01F92CDB7DEB70F90B9
:104A20000F900F900F900F90DF91CF910895CF933B
:104A3000DF9300D000D000D0CDB7DEB726960FB6FA
:104A4000F894DEBF0FBECDBFDF91CF910895CF9315
:104A5000DF93C091230380912403C817A1F0D0E015
:104A6000CE0166E070E00E947930FC01EB5DFC4F06
:104A70004081518162817381848195810E941725D3
:104A80002196C770E8CFDF91CF91089540915503EB
:104A900050915603609157037091580380915903C8
:104AA00090915A030C9417251F93CF93DF93809115
:104AB0005A0382958F7009F05CC080915703882358
:104AC00009F457C02091230310912403C09155038A
:104AD000D0915603A0915803B091590381E0CF3F84
:104AE00009F080E0482F211709F443C0109721F006
:104AF000DF3F21F080E003C081E001C0842F30E07F
:104B000080FD33C0C90166E070E00E947930FC018D
:104B1000EB5DFC4F81818D1328C080818C1325C0F3
:104B20008281811122C0838194818A1B9B0B883CE6
:104B30009105D8F480915A038F70806180935A0355
:104B4000C90166E070E00E947930FC01E65DFC4F2F
:104B500090819F709061908385E593E00E94812110
:104B6000DF91CF911F910C9427252F5F3F4F277026
:104B7000BACFDF91CF911F9108959F92AF92BF92CC
:104B8000CF92DF92EF92FF920F931F93CF93DF9319
:104B9000CDB7DEB761970FB6F894DEBF0FBECDBFBD
:104BA0008C0185E0F801DE011D9601900D928A9539
:104BB000E1F7F80140812181F280C380D480909197
:104BC0005503309156036091580370915903611554
:104BD000710531F03F3F31F481E09F3F19F403C08C
:104BE00081E001C080E0F82FF1709F2E80FD59C157
:104BF00085E5A82E83E0B82EE0905703F601E61B6A
:104C0000F70BEE2009F4EDC080915A03582F507F26
:104C1000E83CF10508F0A7C0511156C0231313C09A
:104C2000491311C0EF2CF1100EC08F70806180937A
:104C30005A030E944625C5010E94812180915A0392
:104C4000F801858364C1C114D10431F02F3F31F4E0
:104C500081E04F3F19F403C081E001C080E080FD96
:104C600003C081E08F2502C080E090E0F82FF17052
:104C7000EF2E80FF1FC0E091230330912403E31740
:104C800009F421C1F0E0CF0166E070E00E947930C4
:104C9000DC01AB5DBC4F11968C911197281307C0B6
:104CA0008C91481304C012968C91F81203C031966F
:104CB000E770E5CFEF2CFF2009F429C180915A035A
:104CC000816080935A0364C0231306C0491304C053
:104CD000F11002C0F801A9C04D872E87FF867C2DF8
:104CE000D98AC88A522F6F2D89890E94B9248823B6
:104CF000A1F1FF2091F120915A03822F82958F70AC
:104D000090E0029774F08091550390915603988734
:104D10008F831986DB86CA862C87CE0107960E9470
:104D2000812186E0F801A5E5B3E001900D928A9516
:104D3000E1F70E9454250E94462512C0231751F125
:104D40004D872E87FF867C2DD98AC88A522F6F2DDA
:104D500089890E94B92481112CC0C8010E94812137
:104D6000EE24E394D4C05111E9CF7C2DD98AC88AAE
:104D7000522F6F2D89890E94082585E593E00E94B6
:104D8000812186E0F50111928A95E9F70E94462576
:104D9000E12CBDC04913D4CFF110D2CFF8018583E7
:104DA000C8010E94812186E0F50111928A95E9F7F8
:104DB000AEC0FF2091F220915A03822F82958F700E
:104DC00090E002970CF4ADCF80915503909156037B
:104DD0009A8389831B82DD82CC822E83CE01019649
:104DE0009ECFE83CF10508F04CC0EF2CFF2009F401
:104DF000B4CF231330C049132EC020915A0320FD95
:104E000021C0822F82958F70482F50E041155105A7
:104E1000C9F0F80125834F30510541F08F5F982F7D
:104E20009295907F822F8F70892B8583C8010E9475
:104E3000812186E0F801A5E5B3E001900D928A9505
:104E4000E1F72CC086E0F801A5E5B3E001900D92F2
:104E50008A95E1F75CC04D872E87FF867C2DD98A25
:104E6000C88A522F6F2D89890E94B924811159CF88
:104E700080915A03816080935A03C8010E94812166
:104E800046C07C2DD98AC88A522F6F2D89890E94ED
:104E9000082586E0F50111928A95E9F70E944625DA
:104EA00036C0FF2009F459CF4D872E87FF867C2D11
:104EB000D98AC88A522F6F2D89890E94B9248823E4
:104EC00009F44BCF2ECF7C2DD98AC88A522F6F2D53
:104ED00089890E94F929292F22952F70223028F4E0
:104EE0009F7039F0811105C00BC0243028F49F70E9
:104EF00049F4805E883020F0C8010E9481219E2CF8
:104F0000E92C05C0F8019581907F99F7F9CF8E2D96
:104F100061960FB6F894DEBF0FBECDBFDF91CF9183
:104F20001F910F91FF90EF90DF90CF90BF90AF90C7
:104F30009F900895CF93DF93CDB7DEB72C970FB630
:104F4000F894DEBF0FBECDBF4F83588769877A873D
:104F50008B879C87CE0107960E94BD258823D1F0C0
:104F60009F8188852A853B85232B31F08F3F31F443
:104F700081E09F3F19F403C081E001C080E080FD23
:104F80006FC04F81588569857A858B859C850E9485
:104F9000172566C086E0FE013796DE011196019066
:104FA0000D928A95E1F7FF81E8856A857B85611519
:104FB000710531F0EF3F31F481E0FF3F19F403C098
:104FC00081E001C080E080FD4BC08091240390E02F
:104FD0009C012F5F3F4F277033274091230350E000
:104FE0002417350709F443C0F983EA837D836C8372
:104FF00066E070E00E947930DC01AB5DBC4F96E06A
:10500000FE01319601900D929A95E1F720932403C9
:105010000E94272525C090E066E070E00E9479306C
:105020008B5D9C4F0E94BD25882371F180912303E5
:1050300090E066E070E00E947930FC01EB5DFC4F8F
:105040004081518162817381848195810E941725FD
:105050008091230390E00196877099278093230322
:1050600080912303909124038913D5CF0DC00E9412
:105070007D211092240310922303E5E5F3E086E0FE
:10508000DF011D928A95E9F72C960FB6F894DEBFE2
:105090000FBECDBFDF91CF910895DF92EF92FF92C7
:1050A0000F931F93CF93DF93FC01892B09F488C0E2
:1050B000E12CF12CDD24D394EF01219684918537E6
:1050C00009F460C058F4843708F04EC0843008F00A
:1050D00068C08130D1F0823071F172C0883709F434
:1050E0005BC050F4863709F453C0873709F068C0B5
:1050F0008E2D0E94362B52C09CE7980F903708F0F7
:105100005FC08F770E9435214EC08F010E5F1F4F09
:10511000FE01849190E2980F983050F48770FD2D35
:1051200001C0FF0F8A95EAF78F2F0E943C2B15C014
:105130000E94762014C08F010E5F1F4FFE018491E4
:1051400090E2980F983068F48770FD2D01C0FF0F32
:105150008A95EAF78F2F0E94422B0E94632BE80169
:1051600022C00E943521FBCFCF010296FE01C491DF
:10517000CC2361F0EFE9FFE03197F1F700C00000C8
:10518000C150F6CFCF010296FE01F490EC010BC0A6
:105190000E94262BE82E07C00E94392B0E94632B09
:1051A00002C00E9476208F2D882341F0EFE9FFE0B6
:1051B0003197F1F700C000008150F6CFFE017CCF9F
:1051C000DF91CF911F910F91FF90EF90DF900895A5
:1051D0006093DB037093DC038093DD039093DE0325
:1051E0000C94C52B08950F931F930091DF0310912A
:1051F000E0032091E1033091E203602B712B822BBD
:10520000932B6093DF037093E0038093E10390930B
:10521000E2031F910F910C94C42B0F931F930091E5
:10522000DF031091E0032091E1033091E20360235A
:105230007123822393236093DF037093E0038093B1
:10524000E1039093E2031F910F910C94C42B0F93F1
:105250001F930091DF031091E0032091E10330914F
:10526000E20360277127822793276093DF037093FF
:10527000E0038093E1039093E2031F910F910C945C
:10528000C42B60E070E0CB010C94E8280F931F93CF
:1052900041E050E060E070E08A019B0104C0000F33
:1052A000111F221F331F8A95D2F7C901B8011F9120
:1052B0000F910C94E8280F931F9341E050E060E0B9
:1052C00070E004C0440F551F661F771F8A95D2F700
:1052D0008091DB039091DC03A091DD03B091DE03AC
:1052E0008A019B01082B192B2A2B3B2BC901B801E2
:1052F0001F910F910C94E8280F931F9341E050E009
:1053000060E070E004C0440F551F661F771F8A9548
:10531000D2F740955095609570958091DB03909100
:10532000DC03A091DD03B091DE038A019B01082319
:1053300019232A233B23C901B8011F910F910C9413
:10534000E8280F931F9341E050E060E070E004C054
:10535000440F551F661F771F8A95D2F78091DB0394
:105360009091DC03A091DD03B091DE038A019B01E3
:10537000082719272A273B27C901B8011F910F9138
:105380000C94E8280F931F930091DB031091DC032A
:105390002091DD033091DE03602B712B822B932B48
:1053A0001F910F910C94E8280F931F930091DB033A
:1053B0001091DC032091DD033091DE036023712323
:1053C000822393231F910F910C94E8280F931F932E
:1053D0000091DB031091DC032091DD033091DE03AB
:1053E00060277127822793271F910F910C94E8283B
:1053F00008958F929F92AF92BF92DF92EF92FF92A9
:105400000F931F93CF93DF9300D000D01F92CDB79F
:10541000DEB76B837C838D838A018C819D81892B90
:1054200031F01F3F31F481E04F3F19F403C081E0B8
:1054300001C080E080FF03C080E090E054C08B8119
:10544000882309F43DC08090DB039090DC03A0909A
:10545000DD03B090DE038091DF039091E003A09123
:10546000E103B091E203882A992AAA2ABB2A2FE1F4
:10547000E22EF12CD501C4010E2C04C0B695A795DF
:10548000979587950A94D2F780FD06C081E0E81AC7
:10549000F10880F7D12C07C0DE2CB8018E2D0E94B8
:1054A000410C019799F3E12FF0E094E0EE0FFF1F1C
:1054B0009A95E1F7E55AFC4FE00FF11DD0820CC040
:1054C000E12FF0E084E0EE0FFF1F8A95E1F7E55A47
:1054D000FC4FE00FF11DD08009831A8369817A8126
:1054E0008D2D0E94410C0F900F900F900F900F90F8
:1054F000DF91CF911F910F91FF90EF90DF90BF90C0
:10550000AF909F908F90089590911101992379F118
:1055100090911201992359F1982F96959695969509
:105520009F31A1F0E0911301F0911401E90FF11DF9
:10553000877021E030E0A90102C0440F551F8A9511
:10554000E2F7CA019181892B818308959091060425
:1055500090FF29C01F928F938AED97E09F938F93BE
:105560000E9436050F900F900F900F900895209194
:10557000130130911401F90132969FEF40E05191EF
:10558000851789F09F3F19F4511101C0942F4F5F87
:105590004E31A9F79F3F39F0F901E90FF11D97FD51
:1055A000FA9582830895089590911101992381F1CC
:1055B00090911201992361F1982F96959695969561
:1055C0009F31A9F0E0911301F0911401E90FF11D51
:1055D000877021E030E0A90102C0440F551F8A9571
:1055E000E2F7CA0180959181892381830895909182
:1055F000060490FF1CC01F928F938CEB97E09F9343
:105600008F930E9436050F900F900F900F90089582
:10561000E0911301F09114019F01225E3F4F9281AE
:10562000891301C012823196E217F307C1F708957A
:1056300081E090E0E0911301F0911401E80FF91F6F
:105640001082019680329105A9F708958091050492
:10565000089590910504892B809305040895809501
:10566000909105048923809305040895809305048F
:10567000089510920504089590910404892B809355
:105680000404089580959091040489238093040470
:1056900008951092040408958093E30308951092EE
:1056A000E30308958091130190911401FC01319658
:1056B0009C01205E3F4F80E0919191118F5FE21736
:1056C000F307D1F70895E0911301F091140180914F
:1056D00005048083E0911301F09114019081809181
:1056E0000404892B80838091E303882361F0E09197
:1056F0001301F09114019081892B80830E94522B19
:1057000081111092E30380911301909114010C9484
:10571000771E90937F0180937E0108958295982F44
:105720009373292F220F220F982F9C7C9695969584
:10573000922B892F8575880F9A7A9695892B0895D3
:10574000CF93DF93D92F0E948E2BC82F8D2F0E94CD
:105750008E2B2C2F30E0322F2227A901482BCA0193
:10576000DF91CF91089508950895CF93DF9300D0EE
:1057700000D01F92CDB7DEB70F900F900F900F9013
:105780000F90DF91CF910895089508950C94E41F30
:1057900080E0089583B7817F8C6083BF83B7816089
:1057A00083BF7894889583B78E7F83BF0895CF9306
:1057B0000E942E200E94EC150E942F20C0E08C2F0A
:1057C0000E94360C892B29F4CF5FC830C1F780E0E6
:1057D00001C081E0CF9108950E943F0C0C947D217F
:1057E0001F920F920FB60F9211248F939F93AF9336
:1057F000BF938091070490910804A0910904B0918F
:105800000A044196A11DB11D8093070490930804DA
:10581000A0930904B0930A04BF91AF919F918F9117
:105820000F900FBE0F901F90189582E084BD93E0FB
:1058300095BD9AEF97BD80936E0008952FB7F894A9
:105840008091070490910804A0910904B0910A0482
:105850002FBF08952FB7F894609107047091080442
:105860008091090490910A042FBF08959C014FB7BD
:10587000F8948091070490910804A0910904B091D4
:105880000A044FBF821B930B089578941F920F92C6
:105890000FB60F9211248F939F93AF93BF93809174
:1058A000070490910804A0910904B0910A0401969C
:1058B000A11DB11D8093070490930804A0930904CF
:1058C000B0930A04BF91AF919F918F910F900FBE3B
:1058D0000F901F9018950E943D1DF89487E797E759
:1058E000909301088093000887E090EBDC0180939F
:1058F000210490932204A0932304B09324049CE0F9
:1059000088E10FB6F894A895809360000FBE90933D
:105910006000FFCF80E090E00895089580910D042D
:1059200080FF0CC08091180190E065E070E00E945B
:10593000793095958795959587952EC081FF0AC0FA
:105940008091180190E065E070E00E9479309595B3
:10595000879522C082FF08C08091180190E065E021
:1059600070E00E94793018C020910E042223D9F0F3
:1059700030911701231780F78091180190E065E0BE
:1059800070E00E947930622F70E00E947930632FBE
:1059900070E00E948A30CB018038910538F400977E
:1059A00039F481E005C085E090E008958FE708951F
:1059B000089580910D0480FF08C06091160170E089
:1059C000759567957595679523C081FF06C06091B1
:1059D000160170E0759567951BC082FF04C0609149
:1059E000160170E012C060910E046623A9F02091A8
:1059F00015016217A0F78091160170E090E00E94F7
:105A00007930622F70E00E948A306038710540F46E
:105A10006115710519F406C061E070E0862F0895E4
:105A20008FE7089581E00895803F21F40E948E2C35
:105A3000819504C0813F29F40E948E2C809311042B
:105A40000895823F21F40E948E2C819504C0833FEB
:105A500029F40E948E2C809310040895893F19F434
:105A60000E94D92C05C08A3F31F40E94D92C81951F
:105A70008093120408958B3F21F40E94D92C8195C4
:105A800004C08C3F29F40E94D92C809313040895FC
:105A9000843F21F480910F04816017C0853F21F479
:105AA00080910F04826011C0863F21F480910F0421
:105AB00084600BC0873F21F480910F04886005C08B
:105AC000883F31F480910F04806180930F04089522
:105AD0008D3F21F480910D0481600BC08E3F21F435
:105AE00080910D04826005C08F3F29F480910D04E0
:105AF000846080930D040895803F39F480911104EF
:105B000087FF6CC01092110469C0813F29F4809115
:105B100011041816BCF362C090911004823F29F45E
:105B200097FF5CC01092100459C0833F19F41916F6
:105B3000CCF354C0893F41F48091120418160CF044
:105B40004DC0109212044AC08A3F29F48091120479
:105B500087FF44C0F6CF8B3F39F48091130487FF51
:105B60003DC0109213043AC08C3F29F48091130475
:105B70001816BCF333C0843F21F480910F048E7F4C
:105B800017C0853F21F480910F048D7F11C0863F9F
:105B900021F480910F048B7F0BC0873F21F480910B
:105BA0000F04877F05C0883F31F480910F048F7EFA
:105BB00080930F0413C08D3F21F480910D048E7FDC
:105BC0000BC08E3F21F480910D048D7F05C08F3F67
:105BD00029F480910D048B7F80930D048091100433
:105BE00081110EC08091110481110AC080911204AC
:105BF000811106C080911304811102C010920E041D
:105C000008958091060483FF7EC08FE198E00E9492
:105C10009D0480910F041F928F938AE198E09F93D7
:105C20008F930E94360588E198E00E949D04809140
:105C30001004282F082E000C330B3F938F9385E11F
:105C400098E09F938F930E94360583E198E00E942D
:105C50009D0480911104282F082E000C330B3F93D4
:105C60008F9380E198E09F938F930E9436058EE09A
:105C700098E00E949D0480911204282F082E000CA9
:105C8000330B3F938F938BE098E09F938F930E9409
:105C9000360589E098E00E949D0480911304282F26
:105CA000082E000C330B3F938F9386E098E09F9370
:105CB0008F930E94360583E098E00E949D048091B6
:105CC0000E041F928F9380E098E09F938F930E9421
:105CD00036058EEF97E00E949D0480910D041F927F
:105CE0008F938BEF97E09F938F930E94360588EFF9
:105CF00097E00E949D048DB79EB74C960FB6F8941E
:105D00009EBF0FBE8DBF8FE094E00E94C01E0E9418
:105D10001E2C90930C0480930B0408951F93CF9333
:105D2000DF9380910B0490910C040E94362CFC01AF
:105D300020910E04222321F08091190190E007C0E8
:105D400080911A0190E06AE070E00E947930E817D3
:105D5000F90708F485C080911004C0911104D09116
:105D6000120410911304811107C0C11175C0D11123
:105D700073C0111171C074C02F3F19F02F5F2093B1
:105D80000E04181624F40E948E2C80931004809127
:105D9000100487FF05C00E948E2C8195809310040B
:105DA0001C1624F40E948E2C8093110480911104FF
:105DB00087FF05C00E948E2C81958093110460910D
:105DC0001004662331F1C0911104CC2311F1062E89
:105DD000000C770B880B990B0E94782F23E333E399
:105DE00043E35FE30E94DC2F0E94402F6093100486
:105DF0006C2FCC0F770B880B990B0E94782F23E325
:105E000033E343E35FE30E94DC2F0E94402F609363
:105E100011041D1624F40E94D92C80931204809141
:105E2000120487FF05C00E94D92C8195809312042B
:105E3000111624F40E94D92C80931304809113042A
:105E400087FF05C00E94D92C819580931304DF91B0
:105E5000CF911F910C94012E2F3F09F08FCFA0CF2F
:105E6000DF91CF911F910895EFE0F4E085E0DF012D
:105E70001D928A95E9F710920E0410920D04089570
:105E80000E94472F6894B1110C94D62F08950E9458
:105E9000BB2F88F09F5798F0B92F9927B751B0F0D2
:105EA000E1F0660F771F881F991F1AF0BA95C9F79E
:105EB00014C0B13091F00E94D52FB1E008950C9438
:105EC000D52F672F782F8827B85F39F0B93FCCF3EB
:105ED000869577956795B395D9F73EF4909580951B
:105EE000709561957F4F8F4F9F4F0895E89409C03B
:105EF00097FB3EF490958095709561957F4F8F4FFD
:105F00009F4F9923A9F0F92F96E9BB279395F69512
:105F1000879577956795B795F111F8CFFAF4BB0F90
:105F200011F460FF1BC06F5F7F4F8F4F9F4F16C0F4
:105F3000882311F096E911C0772321F09EE8872F7E
:105F4000762F05C0662371F096E8862F70E060E03A
:105F50002AF09A95660F771F881FDAF7880F9695B3
:105F6000879597F9089557FD9058440F551F59F09C
:105F70005F3F71F04795880F97FB991F61F09F3F36
:105F800079F087950895121613061406551FF2CF5F
:105F90004695F1DF08C0161617061806991FF1CFAF
:105FA00086957105610508940895E894BB276627D6
:105FB0007727CB0197F908950E94EE2F0C94683053
:105FC0000E945A3038F00E94613020F0952311F081
:105FD0000C9451300C9457300C94D62F0E94B32F50
:105FE00078F39923C9F35523B9F3950F50E0551F62
:105FF000AA27EE27FF27BB2700240894679520F4E3
:10600000E20FF31FB41F0A1E220F331F441FAA1FE3
:106010006695A9F7779530F4F30FB41F0A1E121E88
:1060200008F46395330F441FAA1F221F769599F732
:10603000879520F4B40F0A1E121E631F440FAA1F77
:10604000221F331F8695A9F7862F712D602D1124ED
:106050009F5750409AF0F1F088234AF0EE0FFF1F4F
:10606000BB1F661F771F881F91505040A9F79E3FA6
:10607000510580F00C9451300C94D62F5F3FE4F31F
:10608000983ED4F3869577956795B795F795E795FC
:106090009F5FC1F7FE2B880F911D9695879597F905
:1060A000089597F99F6780E870E060E008959FEF9A
:1060B00080EC089500240A9416161706180609069F
:1060C000089500240A94121613061406050608956E
:1060D000092E0394000C11F4882352F0BB0F40F4F6
:1060E000BF2B11F460FF04C06F5F7F4F8F4F9F4F36
:1060F00008950024552704C0080E591F880F991FC2
:10610000009729F076956795B8F37105B9F7802D5A
:10611000952F089597FB072E16F4009407D077FD6E
:1061200009D00E94A43007FC05D03EF490958195DB
:106130009F4F0895709561957F4F0895EE0FFF1F53
:106140000590F491E02D0994AA1BBB1B51E107C0F7
:10615000AA1FBB1FA617B70710F0A61BB70B881FF7
:10616000991F5A95A9F780959095BC01CD01089586
:04617000F894FFCFD1
:1061740005EA010000FF1816BA168B164F161B16F7
:10618400010101E4032808140A321E5F5A31353034
:10619400005F3F3F3F3F005F4154383400415400AB
:1061A4005854005445524D494E414C004E4F4E45B3
:1061B400004D4F55534500494E54454C4C49004CF5
:1061C4004F474954454348004558504C4F52455257
:1061D4000044454641554C5400397F222607A70602
:0E61E40085062A0643065C0600080004000239
:106800008800EA44E944E244040005000600070069
:10681000080009000A000B000C000D000E000F001C
:1068200010001100120013001400150016001700CC
:10683000180019001A001B001C001D001E001F007C
:10684000200021002200230024002500260027002C
:10685000280029002A002B002C002D002E002F00DC
:10686000300031003200330034003500360037008C
:10687000380039003A003B003C003D003E003F003C
:1068800040004100420043004400450046004700EC
:10689000480049004A004B004C004D004E004F009C
:1068A000500051005200530054005500560057004C
:1068B000580059005A005B005C005D005E005F00FC
:1068C0006000610062006300640065A185006700EC
:1068D000680069006A006B006C006D006E006F005C
:1068E0007000710072007300890087008A008B00BD
:1068F000E000E100E200E300E400E500E600E7007C
:106900000100010001000100EA4401000100E2442D
:106910000100010001000100460001004A004B0097
:10692000010001004700480001000100E9440100A6
:106930000100010001000100010001003A003B00DC
:106940003C003D003E003F0040004100420043004B
:10695000010035004C0039000100440045005200A0
:1069600049000100010050004F0029004D004E0079
:1069700051000100010001000100010001000100BF
:1069800001000100010001000100010001000100FF
:1069900001000100010001000100010001004D00A3
:1069A0004A004E004B0001000100010001000100FF
:1069B00001000100010001000100010001000100CF
:1069C00001000100010001000100010001000100BF
:1069D00001000100010001000100010001000100AF
:1069E0000100010001000100490001000100010057
:1069F000010001000100010001000100010001008F
:00000001FF
